:020000040000FA
:100000001202040000000000A60A0000A60A000078
:10001000A60A0000A60A0000A60A0000A60A000020
:10002000A60A0000A60A0000A60A0000A60A000010
:10003000A60A0000A60A0000A60A0000A60A000000
:10004000A60A000024060000A60A0000A60A000076
:10005000A60A0000A60A0000A60A0000A60A0000E0
:10006000A60A0000A60A0000A60A0000A60A0000D0
:10007000A60A0000A60A0000A60A0000A60A0000C0
:10008000A60A0000A60A0000A60A0000A60A0000B0
:10009000A60A0000A60A0000FA030000A60A000053
:1000A000A60A0000A60A0000A60A0000A60A000090
:1000B000A60A0000A60A0000A60A0000A60A000080
:1000C000A60A0000A60A0000A60A0000A60A000070
:1000D000A60A0000A60A0000A60A0000A60A000060
:1000E000A60A0000A60A0000A60A0000A60A000050
:1000F000A60A0000A60A0000A60A0000A60A000040
:10010000A60A0000A60A0000A60A0000A60A00002F
:10011000A60A0000A60A0000A60A0000A60A00001F
:10012000A60A0000A60A0000A60A0000A60A00000F
:10013000A60A0000A60A0000A60A0000A60A0000FF
:10014000A60A0000A60A0000A60A0000A60A0000EF
:10015000A60A0000A60A0000A60A0000A60A0000DF
:10016000A60A0000A60A0000A60A0000A60A0000CF
:10017000A60A0000A60A0000A60A0000A60A0000BF
:10018000A60A0000A60A0000A60A0000A60A0000AF
:10019000A60A0000A60A0000A60A0000A60A00009F
:1001A000A60A0000A60A0000A60A0000A60A00008F
:1001B000A60A0000A60A0000A60A0000A60A00007F
:1001C000A60A0000A60A0000A60A0000A60A00006F
:1001D000A60A0000A60A0000A60A0000A60A00005F
:1001E000A60A0000A60A0000A60A0000A60A00004F
:1001F000A60A0000A60A0000A60A0000A60A00003F
:10020000FFFFFF00FFFFFF00A60A0000A60A000094
:10021000A60A0000A60A0000A60A0000A60A00001E
:10022000A60A0000A60A0000A60A0000A60A00000E
:10023000A60A0000A60A0000A60A0000A60A0000FE
:10024000A60A000024060000A60A0000A60A000074
:10025000A60A0000A60A0000A60A0000A60A0000DE
:10026000A60A0000A60A0000A60A0000A60A0000CE
:10027000A60A0000A60A0000A60A0000A60A0000BE
:10028000A60A0000A60A0000A60A0000A60A0000AE
:10029000A60A0000A60A0000FA030000A60A000051
:1002A000A60A0000A60A0000A60A0000A60A00008E
:1002B000A60A0000A60A0000A60A0000A60A00007E
:1002C000A60A0000A60A0000A60A0000A60A00006E
:1002D000A60A0000A60A0000A60A0000A60A00005E
:1002E000A60A0000A60A0000A60A0000A60A00004E
:1002F000A60A0000A60A0000A60A0000A60A00003E
:10030000A60A0000A60A0000A60A0000A60A00002D
:10031000A60A0000A60A0000A60A0000A60A00001D
:10032000A60A0000A60A0000A60A0000A60A00000D
:10033000A60A0000A60A0000A60A0000A60A0000FD
:10034000A60A0000A60A0000A60A0000A60A0000ED
:10035000A60A0000A60A0000A60A0000A60A0000DD
:10036000A60A0000A60A0000A60A0000A60A0000CD
:10037000A60A0000A60A0000A60A0000A60A0000BD
:10038000A60A0000A60A0000A60A0000A60A0000AD
:10039000A60A0000A60A0000A60A0000A60A00009D
:1003A000A60A0000A60A0000A60A0000A60A00008D
:1003B000A60A0000A60A0000A60A0000A60A00007D
:1003C000A60A0000A60A0000A60A0000A60A00006D
:1003D000A60A0000A60A0000A60A0000A60A00005D
:1003E000A60A0000A60A0000A60A0000A60A00004D
:1003F000A60A0000A60A0000A60A0000A60A00003D
:100400001C1A000016140000081200000604000068
:10041000100E00000C0A0000020000002826000058
:10042000242200004507A90000002000403A88006F
:100430002FA2200000FF2000000188000000000023
:1004400081E0A80000002000A00188004440A8002E
:10045000C4A2EF00CCA2EF00CCE2A800CD42A800DD
:10046000CD62A800CEE2A900CF42A900CF62A900C8
:10047000C022EF00C822EF00C0E2A8006F20A80051
:100480000060FE0060012000B00C8800000D8800B4
:10049000500D8800C0002100900C8800E00C8800FE
:1004A000300D8800900B20006008880011E1A80042
:1004B0000060FE000000EB00100009000060FE007C
:1004C0000000E900FCFF3A00C2E2AE00FEFF370088
:1004D0002609020000000000004088002080200063
:1004E0004004FC000F0109000018EB00F0FF27009A
:1004F000504088000060FE00700020000008E3000B
:10050000010039000028EF00004080000060010079
:1005100009003700050037001F0037004A00370088
:1005200048003700710037008B0037001E08A80014
:100530005408A8008A08A800E0282800B0408800D5
:10054000E051280060428800D07A280010448800DA
:10055000100020009040880040428800F04388004E
:10056000A04088005042880000448800C00120005C
:100570008040880030428800E0438800008B2000E3
:100580003500090030F0A000B1E8A900E1E8A900B9
:1005900011E9A900AD00370000002000704088007C
:1005A0007023200020428800E0462000D0438800CD
:1005B000A0CE2500B0408800F0FF250060428800F2
:1005C000701C260010448800100020009040880015
:1005D00040428800F0438800A040880050428800D4
:1005E0000044880040002000804088005000200027
:1005F0003042880060002000E0438800008B20002B
:100600003500090030F0A000B1E8A900D5E8A90044
:10061000F9E8A9001E28A8005428A8008A28A800E4
:1006200010002000D04088008042880030448800BC
:1006300010002000E040880090428800404488007C
:10064000820037008A08A8000268A8000000200085
:100650007040880020428800D043880000002100BC
:10066000B0408800F0FF2F0060428800F0FF2F00AC
:10067000104488001000200090408800F00F2000F7
:100680004042880000022000F0438800F00F200064
:10069000A040880000002000504288001000200088
:1006A00000448800100020008040880000002000E6
:1006B0003042880080002000E0438800C091200084
:1006C0003500090030F0A0001DE9A90041E9A900AA
:1006D00065E9A9008A28A80010002000304488009D
:1006E0000000200040448800580037000268A8003D
:1006F000000020007040880020428800D04388001D
:10070000F0FF2000B0408800F0FF2F00604288001A
:10071000F0FF2F0010448800100020009040880057
:10072000F00F20004042880010002000F0438800B5
:10073000F00F2000A04088000000200050428800F8
:10074000004488000000200080408800304288007B
:10075000E04388003D003700000020007040880022
:10076000002020002042880000402000D043880064
:10077000F0FF2F00B04088006042880010448800DD
:10078000100020009040880040428800F04388001C
:10079000A04088005042880000448800E00020000B
:1007A0008040880030428800E0438800008B2000B1
:1007B0003500090030F0A000B1E8A900D5E8A90093
:1007C000F9E8A9001E28A8005428A8008A28A80033
:1007D00010002000D040880080428800304488000B
:1007E000C03F2000E04088009042880040448800DC
:1007F000160037008780A9000060FE0040A7A9000E
:1008000005E1A90011E1A90094E0A90084E0A90094
:100810009780A9008780A900C0A2EF00C8A2EF00BE
:10082000C2E2AE00FEFF37000000EB001800090036
:100830000000E900FDFF3A008660A9006320A800DF
:100840009660A8000040FE000000FE000060FE0070
:1008500040A7A80094E0A800F0FF27001008880037
:1008600005E1A8008460AE00FEFF37008460A900A7
:100870005E050200000000000428AF00DEFF370024
:100880000448AE00060037000448A9000028EC0028
:100890000040800002090200000000000CFF370049
:1008A000504080000C28B400EEFF39000268AF0011
:1008B0000F0037000208A800E1802000028B200012
:1008C000A00502000000000041842000428D2000AD
:1008D000A005020000000000A1872000828F2000F8
:1008E000A0050200000000000208A900DDFF37009B
:1008F000E1802000C2912000A0050200000000005D
:100900004184200002942000A005020000000000A5
:10091000A187200042962000A005020000000000F0
:10092000C3912000078B2000298D20000208A80019
:1009300013027800F40FB200A3129000F50FB2007A
:1009400043239000F60FB200B6040200000000003E
:100950000938E100030032008381E8008783E80062
:10096000F3FF37000208A900BEFF37000500E000D2
:1009700004003A00860B7800A6139800C62398005E
:10098000000006006620B800D05088004800DE0055
:10099000C05088004800DD001A2AB5000010200071
:1009A000050050000600B8004800DE00E050880056
:1009B000D05080000500B8004800DE000000EA00CA
:1009C0000010B0000600B8004800DE00F0508800BB
:1009D000D05080000000EA000010B0000500B80010
:1009E0004800DE000000EA000010B0000600B80079
:1009F0004800DE0000518800C05080000060010007
:100A0000050037000B0037001100370017003700D2
:100A10001D0037002300370006007800800B7800A7
:100A200000518000A0139800E0508000C02398007F
:100A300000000600F0508000800B7800060078006F
:100A4000A0139800E0508000C0239800000006002A
:100A5000E0508000800B780006007800A01398001A
:100A600000518000C023980000000600E050800084
:100A7000800B7800F0508000A013980006007800EA
:100A8000C02398000000060000518000800B780011
:100A9000E0508000A013980006007800C023980062
:100AA00000000600860B7800E0508000A01398003C
:100AB000F0508000C023980000000600101680004F
:100AC0000070A30006A8D600418020006C0502003B
:100AD00000000000000006001100A7000800370019
:100AE000F0FF2F00110190000201600003003A00A6
:100AF0001100A000000F2000A000980000000600D8
:100B0000F0FF2F0011019000020160000001690058
:100B100003003A001100A1001120A000000006000F
:100B2000648140001209E900010032000000060063
:100B30001110A000000F2000A00098000000060087
:100B4000608040001000E000020032001008E90060
:100B50000000060041009000EA8140009309400037
:100B6000010031000000060082047800200220000D
:100B70008005410021069000B1069000110490000C
:100B8000F00F200088035000010B90000600A70022
:100B90000200370062054100010037000B057800B4
:100BA000F28240001900780000F0A6000300370030
:100BB000950AE9001A003A0000F0A10000E0A70041
:100BC0000C0037000044E7001AF0A1000C40400080
:100BD0001300390000C0EB0000E0A2000610A600E0
:100BE0000F00370000F0A000E1019000830A7800B8
:100BF0000B003700003CE7001AF0A1000D40500048
:100C0000070031000040EB0000E0A2000610A60043
:100C10000300370000F0A000F1019000830A780083
:100C2000800C78000B48E700000006008582E80091
:100C30008984E8000A85E8000B50E600D9FF3700F8
:100C400002057800D7FF370000A0FE00849FBE0099
:100C5000404C800000600100400037000D0037006C
:100C6000170037008829EF00604C8000A00C880036
:100C700040C02100800C88006050800071508000CE
:100C80002016880061168800D406020000000000CB
:100C90003C003700604C8000400D880040C02100BF
:100CA000200D880080508000915080002016880020
:100CB00061168800DA0602000000000031003700EB
:100CC000604C8000F00C880040C02100D00C8800EF
:100CD000A0508000B1508000201688006116880066
:100CE0008AA9EC00F00F20008A09E3001F003600FB
:100CF00000002000900188000000EB00052020008B
:100D0000018B2000448D2000E29820003540BA007D
:100D1000313178000408E100FCFF3A000520200092
:100D2000418D2000848F2000829B20003540BA0036
:100D3000313178000408E100FCFF3A000520200072
:100D4000818F2000C4912000229E20003540BA00EF
:100D5000313178000408E100FCFF3A008A29EF00F5
:100D60008A29EC0020002000404C880023702800D5
:100D70008A09D40063007800604C8800CE06020027
:100D8000000000008829EC000060FE004F02BE0059
:100D90000080FE0084E0A90000400600E1982000E9
:100DA000C2A0200005003700819B200002A1200086
:100DB00002003700219E200042A12000534C8000F9
:100DC0000401200004097800310078000304E100E8
:100DD0001289D300FCFF39000A0009001209D10072
:100DE0001299EA0004002800040978003100780014
:100DF0000304E1001289D300FCFF39001299EA00D4
:100E00000000060017000000170000001700000097
:100E10001700000017000000170000001700000076
:100E20001700000018000000190000001900000061
:100E30001A0000001B0000001B0000001C00000046
:100E40001D0000001D0000001E0000001F0000002B
:100E50001F00000020000000210000002200000010
:100E600022000000230000002400000024000000F5
:100E700025000000260000002600000027000000DA
:100E80002800000028000000290000002A000000BF
:100E90002B0000002B0000002C0000002D000000A3
:100EA0002D0000002E0000002F0000002F00000089
:100EB000300000003100000031000000320000006E
:100EC0003300000034000000340000003500000052
:100ED0003600000036000000370000003800000037
:100EE00038000000390000003A0000003A0000001D
:100EF0003B0000003C0000003C0000003D00000002
:100F00003E0000003F0000003F00000040000000E5
:100F100041000000410000004200000043000000CA
:100F200043000000440000004500000045000000B0
:100F30004600000047000000480000004800000094
:100F4000490000004A0000004A0000004B00000079
:100F50004C0000004C0000004D0000004E0000005E
:100F60004E0000004F000000500000005100000043
:100F70005100000052000000530000005300000028
:100F8000540000005500000055000000560000000D
:100F900057000000570000005800000059000000F2
:100FA0005A0000005A0000005B0000005C000000D6
:100FB0005C0000005D0000005E0000005E000000BC
:100FC0005F000000600000006000000061000000A1
:100FD0006200000062000000630000006400000086
:100FE000650000006500000066000000670000006A
:100FF0006700000068000000690000006900000050
:101000006A0000006B0000006B0000006C00000034
:101010006D0000006E0000006E0000006F00000018
:1010200070000000700000007100000072000000FD
:1010300072000000730000007400000074000000E3
:1010400075000000760000007700000077000000C7
:101050007800000079000000790000007A000000AC
:101060007B0000007B0000007C0000007D00000091
:101070007D0000007E0000007F0000007F00000077
:10108000800000008100000082000000820000005B
:101090008300000084000000840000008500000040
:1010A0008600000086000000870000008800000025
:1010B00088000000890000008A0000008B0000000A
:1010C0008B0000008C0000008D0000008D000000EF
:1010D0008E0000008F0000008F00000090000000D4
:1010E00091000000910000009200000093000000B9
:1010F000940000009400000095000000960000009D
:101100009600000097000000980000009800000082
:10111000990000009A0000009A0000009B00000067
:101120009C0000009D0000009D0000009E0000004B
:101130009F0000009F000000A0000000A100000030
:10114000A1000000A2000000A3000000A300000016
:10115000A4000000A5000000A5000000A6000000FB
:10116000A7000000A8000000A8000000A9000000DF
:10117000AA000000AA000000AB000000AC000000C4
:10118000AC000000AD000000AE000000AE000000AA
:10119000AF000000B0000000B1000000B10000008E
:1011A000B2000000B3000000B3000000B400000073
:1011B000B5000000B5000000B6000000B700000058
:1011C000B7000000B8000000B900000000000000F7
:1011D000000000000100000002000000020000000A
:1011E00003000000040000000400000005000000EF
:1011F00006000000060000000700000008000000D4
:1012000009000000F10720009101880001E02F0093
:101210008008BB006027EF0061C7A8006047A800F6
:101220000700FC0051052000313B8800A10A200086
:10123000313B880061E7A8000000000000000000CA
:1012400061E7AF00FEFF370000000600F007200056
:101250009001880000E02F001000BA000000060096
:101260000000FE0000080000220200000200000052
:10127000000000000000000000000000000000006E
:10128000000000000000000000000000000000005E
:10129000000000000000000000000000000000004E
:1012A000000000000000000000000000000000003E
:101540000000000000000000000000000040DA0081
:101550000000FE00FFFFFF00FFFFFF00FFFFFF0096
:10156000FFFFFF00FFFFFF00FFFFFF00FFFFFF0087
:10157000FFFFFF00FFFFFF00FFFFFF00FFFFFF0077
:10158000FFFFFF00FFFFFF00FFFFFF00FFFFFF0067
:10159000FFFFFF00FFFFFF00FFFFFF00FFFFFF0057
:0200000401F009
:100000000F000000000000000300000001000000DD
:10001000DB000000C0000000FF00000083000000C3
:040020001F000000BD
:00000001FF
